:105B680001130000B30101020200000301FA04005E
:105B7800FA0500030A0A5A0B001E0C00FA0D00036E
:105B88000E00030F0164100096120132130AFA1472
:105B9800010215010217010A1801FA1905321A0142
:105BA8000A1B01FA1C05321FFFFF20FFFF23011EFD
:105BB8002400642A00FA2B00FA2C50782D003C2E81
:105BC80000462F001E3000643250783432FA350116
:105BD80064360164370150380A643C00643E003C76
:105BE8003F000040FFFF411450420A5A430AC8448C
:105BF80005324500B44600FA4701044802034C0048
:105C0800FA4EFFFF500404510596520A32530B46D0
:105C1800540A96560102570546580002590A465A30
:105C280032FA5B010A5C0A325E000A5F00FE61FF1D
:105C3800FF64FFFF6600026701016A0A3C6B00000F
:105C48006C32967300007400007801327901327E5C
:105C5800FFFF81FFFF84FFFF8500AF8600018700FB
:105C6800FA89010A8A00009900009D0A969E00019F
:105C78009FFFFFFAFAFA0000B301010202000003D5
:105C880001FA0400FA0500030A0A5A0B001E0C0068
:105C9800FA0D00030E00030F016410009612013282
:105CA800130AFA14010215010217010A1801FA1958
:105CB80005321A010A1B01FA1C05321FFFFF20FFDB
:105CC800FF23011E2400642A00FA2B00FA2C5078C6
:105CD8002D003C2E00462F001E30006432507834D0
:105CE80032FA350164360164370150380A643C00E1
:105CF800643E003C3F000040FFFF411450420A5AF6
:105D0800430AC84405324500B44600FA4701024830
:105D180002024C00FA4EFFFF500404510596520A45
:105D280032530B46540A965601015705465800014E
:105D3800590A465A32FA5B010A5C0A325E000A5F67
:105D480000FE61FFFF64FFFF6600026701016A0A47
:105D58003C6B00006C3296730000740000780132CE
:105D68007901327EFFFF81FFFF84FFFF85FFFF86F9
:105D7800FFFF87FFFF8901028A00009900009D0A42
:105D8800969E00019FFFFFFAFAFA0065006F0079FE
:105D98000083008D009700A100AC00B600C000CAC7
:105DA80000D400DE00E800F2005B0063006A0072C5
:105DB800007A008200890091009900A100A800B033
:105DC80000B800BF00C700CF00D600DF00E600EE35
:105DD80000F600400046004C00520059005F006584
:105DE800006B00710077007D00830089008F0095AB
:105DF800009C00A200A800AE00B400BA00C000C613
:0E5E080000CC00D200D900DF00E500EB00F175
:1035E700900042E0D3940440149007B3E0FEA3E0B8
:1035F700FF905B6A125F4FE493F59980129007B3CF
:10360700E0FEA3E0FF905C7E125F4FE493F5999094
:1036170007B3E0FEA3E0FF905B68E493FC740193BB
:10362700FDEFB50507EEB50403754D009007B3121E
:103637005F362285F97285FA737E017F00E5731282
:103647005F28E5722FFF50010E8E598F5A90001395
:10365700E0FCA3E0FDEF2DFDEE3CFC8C5B8D5C22D6
:1036670075A71085F97285FA737E017F00E57312DD
:103677005F28E5722FFF50010E8E598F5A9000D5A3
:10368700E0B40210AC2CAD2DEF2DFDEE3CFC8C5BB5
:103697008D5C8016AE59AF5A900013E0FCA3E0FD95
:1036A700EF2DFDEE3CFC8C5B8D5C22AE59AF5A745E
:1036B700B48E048F05FF125F188C5B8D5CAE59AF1B
:1036C7005A74B48E048F05FF125F438C598D5AE5E7
:1036D7005A4559601374B4C3955AFFE49559FE8E41
:1036E700598F5A785B125F7C22900083E0B4010403
:1036F700C2138002D213900084E0B40104C2148084
:1037070002D2149000C1E075F0DCA4FFAEF0740A99
:103717008E048F05FF125F189007A9ECF0A3EDF058
:10372700A20D401674038C068D07125F28740112D0
:1037370000399007A7EEF0A3EFF07E017F0090001D
:103747007FE0125F289000C2E08E048F05FF125FB2
:1037570018740AFF125F188D5F9000CBE075F0DCDC
:10376700A4FFAEF0740A8E048F05FF125F1890074E
:10377700ADECF0A3EDF09000CDE060139000CDE04C
:10378700F5F0741684FF7E00EF9007B7F08006749B
:10379700649007B7F09000C3E0900067F090010DC8
:1037A700E0900051F090009CE0900053F09000C52D
:1037B700E0900054F0900071E0900055F09000F711
:1037C700E090005AF074E3900066F09000ACE0B42B
:1037D7000B0874E3900066F0805A9000ACE0B419CF
:1037E700129000C2E0905D7D12008CE49390006619
:1037F700F080419000ACE0B41E129000C2E0905DF2
:103807009B12008CE493900066F080289000ACE057
:10381700B428129000C2E0905DC512008CE493902A
:103827000066F0800F9000ACE0B446089000A3E07B
:10383700900066F090006AE0FE9000A9E0B50633BC
:1038470090006CE0FE9000C7E0B5062790006BE0A3
:10385700FE9000D5E0B5061B90006EE0FE90007C60
:10386700E0B5060F90006DE0FE9000B7E06E7003C4
:103877000239BA900042E0C39405500874029000E0
:10388700F8F080149000D5E0600874089000F8F014
:103897008006740A9000F8F090007CE0B40106748A
:1038A700009000E2F090007CE0B402067400900003
:1038B700C7F090007CE0B4030674009000D4F09049
:1038C70000C7E0D39401401474189000FAF0740014
:1038D7009006C1F074009006C2F0800C740090004E
:1038E700FAF074189006C1F09000A9E06014741AF9
:1038F700900090F074009006C9F074009006CAF02A
:10390700800C7400900090F0741A9006C9F0900033
:10391700A9E0B402147419900091F074009006C5E0
:10392700F074009006C6F0800C7400900091F0745B
:10393700199006C5F09000D5E0700E74059006D575
:10394700F074069006D9F0801874009006D5F074CC
:10395700009006D6F074009006D9F074009006DA4D
:10396700F0D2299000A9E090006AF09000D5E0908D
:10397700006BF09000C7E090006CF09000B7E0900B
:10398700006DF090007CE090006EF090007CE0907D
:103997000052F09000B7E0900056F09000D5E0900C
:1039A7000057F09000A9E0900058F09000C7E09011
:1039B7000059F09000DFE0B4011790001F740FF07A
:1039C700A374FFF0900021E4F0A3F074029000DFED
:1039D700F09000DFE0B40341900021E0FEA3E0FF98
:1039E70090001FE0FCA3E0FD125F747410125F28C3
:1039F7007408120039EF900063F0EF700674FF90BF
:103A07000063F074009000DFF0900020E090006405
:103A1700F090001FE0900065F09000377401F0749B
:103A270002900038F07550019000B6E0900039F030
:103A3700900039E0D39402400F900039E0C394021C
:103A4700900039F0D2238002C223900039E0D3944A
:103A570001400890003A7401F08006740290003A21
:103A6700F022C293C294C291C292C287C290E5B5B6
:103A770054EFF5B5E5B554DFF5B5C296C295C2A0CA
:103A8700C297C2A2C2A1E5B554BFF5B5E5B5547F4B
:103A9700F5B5E5B554FBF5B5C215755D469000B9AA
:103AA700E07005756C028003756C037554007553DF
:103AB7000090000874FFF0A374DCF0C21AC21C74F3
:103AC700C8900033F074C8900035F07552007551F6
:103AD70000C20D754600E56EB40903756E00756288
:103AE70000900015E4F0A3F0756F10C218C219908A
:103AF70007A9E0FEA3E0FF7403125F287401120018
:103B0700399007A7EEF0A3EFF0C20275560075557E
:103B17000090000CE4F0A3F0C22A75580075570016
:103B270090007BE075F032A4FDACF090001DECF046
:103B3700A3EDF0C20EC23A2285F97285FA737E01AF
:103B47007F00E573125F28E5722FFF50010E8E5933
:103B57008F5AAC5BAD5CEF2DFDEE3CFC8C5B8D5C56
:103B6700D293D294E55CF5FBE55BF5FCE55CF5E902
:103B7700E55BF5EA9000B7E0B40314D291D292E581
:103B87005CF5EBE55BF5ECE55CF5EDE55BF5EE2269
:103B970075A71085F97285FA737E017F00E57312A8
:103BA7005F28E5722FFF50010E8E598F5A7E017FD5
:103BB700769000F4E0125F28AC59AD5AED2FFFEC78
:103BC7003EFE8E5B8F5CE55CF5FDE55BF5FE9000E8
:103BD70067E4F075A700741290003EF02285F97231
:103BE70085FA737E017F00E573125F28E5722FFF68
:103BF70050010E8E598F5A9007A9E0FCA3E0FDEF04
:103C07002DFDEE3CFC8C5B8D5CE55CF5FDE55BF525
:103C1700FE220563229000B7E0B403539000D5E07D
:103C2700B4012EA2D8B34004C293C287A2D9B3402D
:103C370004C294C290A2DAB34008C291E5B554EF2A
:103C4700F5B5A2DBB34008C292E5B554DFF5B58000
:103C57001CA2D8B34002C293A2D9B34002C294A215
:103C6700DAB34002C291A2DBB34002C292801EA225
:103C7700D8B3400AC2939000D5E06002C287A2D9A8
:103C8700B3400AC2949000D5E06002C290A2DCB3B0
:103C97004004C296C29575D8402285A77175A710B2
:103CA700A2D8B34002C287A2D9B34002C290A2DA17
:103CB700B34006E5B554EFF5B5A2DBB34006E5B56D
:103CC70054DFF5B5A2DCB340089000C3E09000676D
:103CD700F075D8408571A722900047E49364066089
:103CE7000280FE74C89007AFF8E4F0E8A3F075B55A
:103CF7000075840175A70075FFA090003BE4F0757F
:103D0700C91075A70F75A1C775A70075D90075CE1E
:103D17000C75A70F75F1FE75F2FF75F30775F4784B
:103D270075A4BA75A5FF75A60775AE0075AFFF75C3
:103D3700D48175D5FF75D6FF75D7FF75A70075A216
:103D47000175A14775F80975D80075D90475DA09A1
:103D570075DB0975DC0975DD0975DE0975D84075F0
:103D6700A71075D80075D90475DA0975DB0975DCF4
:103D77000975DD0975DE0975D84075A70075E60870
:103D870075E71075BC0175BE0475BD6C75BE07750A
:103D9700BDA075BE0875BD0175BC0075BB1875BCA7
:103DA7002075BA0875E88075D11375A70F75E105F9
:103DB70075E20075C740123A697597007597807468
:103DC7000A125F087597C0E5975420700280F8754E
:103DD7008F0275A700D2AF75980075A90C75A70F4C
:103DE70075AB4375ADFB75AC1E75A71075C9187516
:103DF700CA0075CB0075C80475A700758912758E42
:103E070004758C00758A00C2A9D28C758D00758BDC
:103E170000D2ABD28E75EF0675D944C29974C8F536
:103E2700097508001200E375B5001204E374639086
:103E370007AFF8E4F0E8A3F012036F74C89007AF78
:103E4700F8E4F0E8A3F07464F5097508001200E3DC
:103E5700900052E090007CF0C22090007CE0D39468
:103E6700034006740090007CF090007CE09057803F
:103E7700F82828738028A2B44002D220802075A792
:103E87000F75F30F75A700A2A34002D220800F750C
:0E3E9700A70F75F31775A700A2A44002D22052
:0C578000023E7B023E7D023E85023E960A
:103EA500A220B34066757208E572D3940E5020E5E2
:103EB500729007AFF8E4F0E8A3F012023E7464F5DF
:103EC500097508001200E37872740126F650D9745A
:103ED500029000B8F090007CE0D394034006740093
:103EE50090007CF090007CE090578CF82828738037
:103EF5001674009000E2F0800E74009000C7F08008
:073F05000674009000D4F0E7
:0C578C00023EF4023EF6023EFE023F0622
:103F0C00D21F8064757201E572D394075020E5725C
:103F1C009007AFF8E4F0E8A3F012023E7464F509E0
:103F2C007508001200E37872740126F650D97401FA
:103F3C009000B8F090007CE0D3940340067400909D
:103F4C00007CF090007CE0905798F828287380163D
:103F5C0074009000E2F0800E74009000C7F08006B0
:063F6C0074009000D4F087
:0C579800023F5A023F5C023F64023F6C7B
:103F7200C21F900051E090010DF0900052E09000BD
:103F82007CF0900053E090009CF0900054E0900090
:103F9200C5F0900055E0900071F0900056E090005E
:103FA200B7F0900057E09000D5F0900058E09000F4
:103FB200A9F0900059E09000C7F090005AE09000FC
:103FC200F7F09000C2E07006740A9000C2F0900010
:103FD200A3E0700674E39000A3F09000A9E00490BF
:103FE200006AF01236F0E5B54401F5B574069000AA
:103FF20040F07401900041F07403900043F07405A6
:10400200900044F07430900045F07405900046F042
:10401200900042E0B404067404900046F0740090EC
:104022000047F0740090004CF0740090004DF07462
:104032000190004EF0740090004FF074FF90005019
:10404200F07434900146F0742B900147F074329072
:104052000148F07448900149F0746F90014AF0747D
:104062006D90014BF0746590014CF0742090014DFD
:10407200F0743490014EF0744390014FF0747990D3
:104082000150F0746C900151F07420900152F07460
:1040920044900153F07453900154F09000DEE0908C
:1040A2000063F0900095E0900064F0900096E0903C
:1040B2000065F0A2B6B39211A2B6B39210A2B3B346
:1040C2009212A2B3B3920FA2A4B39226A2B4B39255
:1040D20027A2A3B3922890005FE4F0756E00743AB1
:1040E20090076FF074FD900770F0900060E4F0901C
:1040F20007A9E0FEA3E0FF7403125F287401120017
:10410200399007A7EEF0A3EFF0756D0190003EE441
:10411200F0C225756200C216D217C202757000C2C3
:104122002CD203C22DD204C22ED205C22FD206C275
:1041320030D207C231D208C232D209C233D20AC245
:1041420034D20BC235D20CC221C222C223C224C233
:104152002912009E755E00756A00756000756432F2
:104162007565007566007567007568007569009071
:104172000015E4F0A3F0756B00D2B2D2A4D2B0D293
:10418200B1D2A3D2A7D2A6D2A5D2B790007BE0D358
:1041920094FA400674FA90007BF07E017F00900052
:1041A20065E0125F28900064E02FFF50010E90003E
:1041B2001FEEF0A3EFF0EFD394FFEE940F400790C1
:1041C200001FE4F0A3F0900063E0700674FF90001B
:1041D20063F074009000A2F09000B8E0D394024023
:1041E2000674019000B8F09000B9E07005756C0299
:1041F2008003756C039000BAE0D39401400674000A
:104202009000BAF09000C0E0C3940A5006740A907D
:1042120000C0F09000CAE0700674019000CAF090ED
:1042220000CAE0B4FF0674FE9000CAF09000D1E02C
:10423200D394FE400674FE9000D1F09000F7E0D3D4
:104242009402400674019000F7F090010DE0D394BF
:10425200014006740190010DF074019000D7F074D2
:10426200019000D8F074009000DFF074009000FB21
:10427200F074009000FFF074299006B5F0742A9053
:1042820006B9F074179006BDF0741B9006CDF07459
:104292001C9006D1F0D29C9000AAE0D39404400670
:1042A20074049000AAF09000DCE0D39404400674F9
:1042B200049000DCF0E56FD394104003756F10900A
:1042C20006B6E0D3940C400674009006B6F0900651
:1042D200BAE0D3940C400674009006BAF09006BE81
:1042E200E0D3940C400674009006BEF09006C2E043
:1042F200D3940C400674009006C2F09006C6E0D338
:10430200940C400674009006C6F09006CAE0D3945E
:104312000C400674009006CAF09006CEE0D3940CCE
:10432200400674009006CEF09006D2E0D3940C4082
:104332000674009006D2F09006D6E0D3940C4006A4
:1043420074009006D6F09006DAE0D3940C4006741E
:10435200009006DAF0D2EC75CF01A298B34005C204
:1043620098120616E54D6006A299B3B34002800585
:10437200C299120AB4E54E64016005E54EB4040226
:1043820080D5C28E7E087F00E563125F28E58D75B9
:10439200F008A4FDACF0EF2DFDEE3CFCE58B75F0D2
:1043A2002084FF7E00ED2FFFEC3EFE8E538F54D211
:1043B2008E90009CE0605C900017125F36900017B0
:1043C200E0FCA3E0FD900019E0FAA3E0FBEDB503E9
:1043D20042ECB5023EB21EA20DB3401975E700A22F
:1043E2001EB34008E5B54404F5B58006E5B554FBB7
:1043F200F5B575E710900019E0FEA3E0FF90001BF1
:10440200E0FCA3E0FDEF2DFDEE3CFC900019ECF08A
:10441200A3EDF09000A9E060099000A9E0C3940325
:104422004002806F1229C0A20DB3500990005FE0D4
:10443200C3940740028006900093E0F545E5457578
:10444200F005A4FFAEF09007B1EEF0A3EFF09000FC
:1044520080E0C395604007E55EC3955F5007900713
:10446200B1E4F0A3F0AE2EAF2F9007B1E0FCA3E0D1
:10447200FDEFD39DEE9C4004C2A1800B90005FE053
:10448200C3940A5002D2A19000A9E0B40205A2A1ED
:10449200B392A29000A9E0B4031C122ADBAE2EAFA5
:1044A2002F9007B1E0FCA3E0FDEFD39DEE9C40040A
:1044B200D2A18002C2A1A2B3301201B34041A2B381
:1044C200301201B34039A2B3301401B34024A2B672
:1044D200B3301001B34004B210800BA215B34006F2
:1044E200740590003EF0A2B6B34002D221A214B3EA
:1044F2009212A214B330B301B34004A2149212A2D6
:10450200B6301101B35003024A47A2B6301101B3CB
:104512005003024A47A2B6301301B3500302488B3C
:10452200756D00A2B3B3300F01B34004B20F800B1C
:10453200A215B34006740490003EF0055DA2B330AC
:104542001401B3B35006A215B3B34003024609E502
:104552006CB4032EA22AB34022E55DB40303756C4A
:1045620001E55DC39403500690003E7401F0E55DE1
:10457200D394034006740290003EF0755D01D22A86
:10458200805AE56CB40206756C01755D03E55DB495
:104592000305755D01804590003EE07030E55DC326
:1045A2009403500690003E7401F0E55DD3940340FD
:1045B20006740290003EF0E55DC394035002D225DA
:1045C200E55DD394034002D225C296C2959000B90C
:1045D200E0B40105123A698003755D01A221B3407E
:1045E20006A22392228002B222C221A2B4B34002C6
:1045F200C227A2A4B34002C226A2A3B34002C22889
:10460200A225B34002C225E55DB4025490009CE0AD
:10461200600990009CE0C3943D40028043900017E3
:10462200E0FEA3E0FF90009CE08E048F05FF125F86
:104632001874018C068D0712003990001BEEF0A34E
:10464200EFF090001BE0F8A3E0900019C8F0A3C8B7
:10465200F0900017E4F0A3F0C21EE5B554FBF5B5E7
:10466200AE57AF58AC53AD54EF2DFDEE3CFC8C571A
:104672008D58AE53AF54EFD39DEE9C401190000F76
:10468200E0FAA3E0FBEBC394E8EA9403400280065D
:1046920090000F125F36900008E553F0A3E554F046
:1046A20090000AE553F0A3E554F0AE53AF547412F0
:1046B2008E048F05FF125F188C558D56C28E758D34
:1046C20000758B00756300755401755300D28E908E
:1046D2000008E0FEA3E0FFEF4E600B7C827D4C12EF
:1046E2005E168E518F52AE51AF527428BE00039F98
:1046F2005010E5622FFF50010E74011200398E51E5
:104702008F528552629000C0E0A851B8000DD39537
:10471200524008E55290003DF080099000C0E0143C
:1047220090003DF0E56C60067552007551009000F6
:10473200B7E0B40308900039E0655D6002800BA227
:1047420022B34004D2248002B2249000A9E0600384
:1047520012202BE56EB40903756E00A216B3500643
:10476200A215B3B34003024810900075E0B4017380
:104772009000F7E0B40214120C55900068E075F056
:10478200BEA4FFAEF08E5B8F5C8056E56675F00AC4
:1047920084FF7E0090056F125F4FE0F55A75590055
:1047A200AE59AF5A90009AE0125F2874648E048F5B
:1047B20005FF125F188C5B8D5CE55C90000EF0AE1D
:1047C20059AF5A900073E0125F2874648E048F050B
:1047D200FF125F1874BE8C068D07125F288E5B8FE6
:1047E2005C8017900073E075F0BEA4FFAEF08E5BA4
:1047F2008F5C90009AE090000EF0E560C394CC507C
:1048020006900073E070028003123B3FD216E56C03
:10481200B40106A215B3B340028009756F0190007E
:104822003F7401F0E56C705C9000BCE0600D90009C
:1048320067E0A851B800069552400280299000BC5A
:10484200E0B40208756F03756B00800CC200756BD3
:1048520000900015E4F0A3F0900067E06006740990
:1048620090003EF0801EE55DB4010B756F01900073
:104872003F7401F0800EE55DB40209756F017402A8
:1048820090003FF0A213B39211A213B330B601B35A
:104892005003024A47756D01E5B54401F5B5740749
:1048A20090005FF0A2139211E55DD394474014D2B9
:1048B20015E55DD3944B400B740590003EF0D22574
:1048C200755D469000C4E0B40107E569C3941440E5
:1048D200028009123A69741390003EF0A22C300350
:1048E20001B3501D75E700A22CB34008E5B544089A
:1048F200F5B58006E5B554F7F5B575E710A22C922B
:1049020003A22D300401B3501D75E700A22DB34060
:1049120008E5B54402F5B58006E5B554FDF5B57573
:10492200E710A22D9204A22E300501B3500FA22E41
:10493200B34004D2A08002C2A0A22E9205A22F30C0
:104942000601B3500FA22FB34004D2978002C29740
:10495200A22F9206A230300701B3500FA230B3400B
:1049620004D2A28002C2A2A2309207A23130080170
:10497200B3500FA231B34004D2A18002C2A1A2312E
:104982009208A232300901B3501D75E700A232B37A
:104992004008E5B54440F5B58006E5B554BFF5B528
:1049A20075E710A2329209A233300A01B3501D7585
:1049B200E700A233B34008E5B54480F5B58006E5CB
:1049C200B5547FF5B575E710A233920AA234300BC5
:1049D20001B3500FA234B34004D2878002C287A22F
:1049E20034920BA235300C01B3500FA235B3400400
:1049F200D2908002C290A235920CE569C3944150D4
:104A020009740E90003EF0123A69900046E0FE9062
:104A12000042E004C39E4009900042E0D394064065
:104A22000974FB90003EF0123A6990004BE0601569
:104A320090004BE0FE900045E06E600974FE90002D
:104A42003EF0123A69A225B34004C296C295900084
:104A5200F4E0600CAE51AF527414BE00059F4002E8
:104A6200804890007CE09057A4F8282873803BA2ED
:104A7200B4B35005A227B340028005123B97D22758
:104A82008028A2A3B35005A228B340028005123B9E
:104A920097D2288015A2A4B35005A226B340028063
:0A4AA20005123B97D2268002800027
:1057A400024A6F024A71024A84024A97024AAA02D2
:0257B4004AACFD
:104AAC00A218B3B35008900039E0655D6003024B67
:104ABC008BA201B35006A200B3B34003024B879004
:104ACC0000B7E0B403028003024B5CA20DB3406755
:104ADC00A224B3402D12363AE55CF5FBE55BF5FC00
:104AEC00D293A202B34002D2879000D5E0B4021058
:104AFC00123667E55CF5FBE55BF5FC75A700D28724
:104B0C00803312363AE55CF5EBE55BF5ECD291A21D
:104B1C0002B34006E5B54410F5B59000D5E0B402FB
:104B2C0014123667E55CF5EBE55BF5EC75A700E573
:104B3C00B54410F5B5801712363AE55CF5FBE55B2C
:104B4C00F5FCE55CF5EBE55BF5ECD293D291802BB3
:104B5C0012363AE55CF5FBE55BF5FCD293A202B3A9
:104B6C004002D2879000D5E0B40210123667E55CA3
:104B7C00F5FBE55BF5FC75A700D287C218D219A22C
:104B8C0019B3B3500890003AE0655D6003024C6ABB
:104B9C00A201B35006A200B3B34003024C669000CE
:104BAC00B7E0B403028003024C3BA20DB34067A2F2
:104BBC0024B3402D12363AE55CF5E9E55BF5EAD213
:104BCC0094A202B34002D2909000D5E0B40210122D
:104BDC003667E55CF5E9E55BF5EA75A700D29080F0
:104BEC003312363AE55CF5EDE55BF5EED292A202B6
:104BFC00B34006E5B54420F5B59000D5E0B40214F9
:104C0C00123667E55CF5EDE55BF5EE75A700E5B5ED
:104C1C004420F5B5801712363AE55CF5E9E55BF50D
:104C2C00EAE55CF5EDE55BF5EED294D292802B12C1
:104C3C00363AE55CF5E9E55BF5EAD294A202B340BD
:104C4C0002D2909000D5E0B40210123667E55CF504
:104C5C00E9E55BF5EA75A700D290D218C219E56FA9
:0E4C6C009057B6F82828730250F39000DCE051
:0657B600024C73024C7668
:104C7A009057E9F8282873121B078012121B078025
:0E4C8A000D121B918008121C3D8003121C3D70
:0F57E900024C81024C86024C8B024C90024C9574
:104C9800756F020250F3121D69121E80A23AB340CA
:104CA8000C90009EE0F56B741090003EF090006F41
:104CB800E0256BF5349007A7E0FEA3E0FF740A1225
:104CC8005F2890000AE0FCA3E0FD74098F02FF1240
:104CD8005F188D078C038E048A058B06125E16906A
:104CE80007ABEEF0A3EFF09000C5E0B401087478CC
:104CF800BE00059F4002800D74789007ABF8E4F081
:104D0800E8A3F0801B9007ABE0FEA3E0FF74F0BEC1
:104D180000039F500B74F09007ABF8E4F0E8A3F0A1
:104D2800E53470037534019007ABE0FEA3E0FFE5BE
:104D3800342FFF50010E9007ABEEF0A3EFF0756F24
:054D48000390003FE0B4
:0357BC00024C9EFE
:104D4D009057F8F82828738010A23B4003756F0A1E
:094D5D008007A23B4003756F0BB7
:0957F800024D54024D56024D5FB2
:104D66000250F39006B6E060031221149000F5E0BD
:104D7600B401149000F6E0A851B80004955250070B
:104D8600E55EC3955F40028003024E139000AAE0E1
:104D9600D39402403F90007EE02403A851B800045B
:104DA60095525009900080E0D3956050028008D259
:104DB60001740890003EF090007EE0A851B800050E
:104DC600D39552500B900080E02403C395605002A7
:104DD600C201803990007EE02403A851B8000495F2
:104DE600525007E55EC3955F40028008D201740801
:104DF60090003EF090007EE0A851B80005D3955291
:104E06005009E55F240FC3955E5002C2019000C4AD
:104E1600E07007E569C3941440028002D201A20142
:104E26004005756F04800A756F10900015E4F0A3B5
:104E3600F0A20DB34029E56675F00A84FF7E009066
:104E4600056F125F4FE0C394695005122060800F12
:104E56009007A9E0F8A3E09007A7C8F0A3C8F0025E
:064E660050F39000AAE0E9
:0657BF00024D69024E6874
:104E6C00905801F8282873120D3F8012120D3F80C4
:0E4E7C000D120EED8008120F9F8003120F9F83
:0F580100024E73024E78024E7D024E82024E8797
:104E8A009006BAE060031221F0756F050250F31222
:104E9A0010AB756F069006BEE060031222E0900622
:104EAA00C2E060031223BC0250F390000EE06006D9
:104EBA00A20DB3B34002801D90000EE02529FFAE7B
:104ECA002850010E8E288F29E55DD3940150069053
:104EDA00000EE014F01212F1756F079006C6E0603A
:104EEA00031224989006CAE060031225740250F354
:104EFA009000F7E0B40203120CCD12154E756F083C
:104F0A009006CEE060031226509006D2E0600312AB
:104F1A00272C0250F312190AA218B35005A219B38A
:104F2A0040028004D218D219756F109006D6E0603C
:104F3A00031228089006DAE060031228E40250F30C
:104F4A000250F3900034E0C394465008C296744667
:104F5A00900034F085345A755900900037E0F572A4
:104F6A001236B2E55C900034F0900004E559F0A3E3
:104F7A00E55AF0C21B900070E0FE900034E0C39E38
:104F8A005012900070E0FE900034E0F4042E90007D
:104F9A0034F08012900070E02402FE900034E0F4B5
:104FAA00042E900034F09007ABE0F559A3E0F55ACF
:104FBA00900037E0F5721236B2E55C900033F0905B
:104FCA000000E559F0A3E55AF0C21A900070E0FE1D
:104FDA00900033E0C39E5012900070E0FE900033C0
:104FEA00E0F4042E900033F08012900070E0240266
:104FFA00FE900033E0F4042E900033F0E56CB40127
:10500A0005756F0B8003756F030250F3900036E04D
:10501A00C3944650139000C5E0B40104C2968002BE
:10502A00C2957446900036F085345A75590090003E
:10503A0038E0F5721236B2E55C900036F090000660
:10504A00E559F0A3E55AF0C21D900070E004FE9005
:10505A000036E0C39E5013900070E004FE900036C4
:10506A00E0F4042E900036F08012900070E02403E1
:10507A00FE900036E0F4042E900036F09007ABE084
:10508A00F559A3E0F55A900038E0F5721236B2E508
:10509A005C900035F0900002E559F0A3E55AF0C2A1
:1050AA001C900070E004FE900035E0C39E501390FF
:1050BA000070E004FE900035E0F4042E900035F014
:1050CA008012900070E02403FE900035E0F4042E74
:1050DA00900035F0E56CB40103756C00756F0380C0
:0950EA00088006800480028000A9
:1057C500024E99024EB4024EFA024F1F024F4A0290
:1057D5004F4D0250160250EB0250ED0250EF0250B1
:0457E500F10250F38A
:1050F300900033E0B55D02800302518EA21A406B2B
:10510300900000E0FEA3E0FFEF4E605DAC51AD52B6
:10511300740ABC0033D39D402FAA55AB5674058A3D
:10512300048B05FF125F188D068C07900000E0FCCE
:10513300A3E0FDCFCECF120003740112003990001B
:1051430000EEF0A3EFF08021AE55AF56900000E0E3
:10515300FCA3E0FD120003740A8E048F05FF125FA7
:1051630018900000ECF0A3EDF0D21AAE53AF5490B8
:105173000000E0FCA3E0FDEFC39DEE9C400D123B5D
:10518300E4D296C21A74C8900033F0A21AB3B35093
:1051930007900033E0B55D02800D123BE4D29674B4
:1051A300C8900033F0C21A900034E0B55D0280036A
:1051B300025242A21B406B900004E0FEA3E0FFEF0B
:1051C3004E605DAC51AD52740ABC0033D39D402F89
:1051D300AA55AB5674058A048B05FF125F188D061A
:1051E3008C07900004E0FCA3E0FDCFCECF120003B8
:1051F3007401120039900004EEF0A3EFF08021AEA9
:1052030055AF56900004E0FCA3E0FD120003740ABE
:105213008E048F05FF125F18900004ECF0A3EDF0ED
:10522300D21BAE53AF54900004E0FCA3E0FDEFC3E8
:105233009DEE9C400AC2967446900034F0C21BA2B5
:105243001BB3B35007900034E0B55D02800AC296E9
:105253007446900034F0C21B900035E0B55D0280C7
:1052630003025301A21C406B900002E0FEA3E0FF87
:10527300EF4E605DAC51AD52740ABC0033D39D4018
:105283002FAA55AB5674058A048B05FF125F188D40
:10529300068C07900002E0FCA3E0FDCFCECF120006
:1052A300037401120039900002EEF0A3EFF08021A5
:1052B300AE55AF56900002E0FCA3E0FD120003746C
:1052C3000A8E048F05FF125F18900002ECF0A3ED25
:1052D300F0D21CAE53AF54900002E0FCA3E0FDEF0C
:1052E300C39DEE9C4018123BE49000C5E0B401045A
:1052F300D2968002D295C21C74C8900035F0A21CCD
:10530300B3B35007900035E0B55D028018123BE45B
:105313009000C5E0B40104D2968002D29574C8907F
:105323000035F0C21C900036E0B55D0280030253E5
:10533300CBA21D406B900006E0FEA3E0FFEF4E60A2
:105343005DAC51AD52740ABC0033D39D402FAA55B6
:10535300AB5674058A048B05FF125F188D068C0704
:10536300900006E0FCA3E0FDCFCECF120003740152
:10537300120039900006EEF0A3EFF08021AE55AF96
:1053830056900006E0FCA3E0FD120003740A8E04AD
:105393008F05FF125F18900006ECF0A3EDF0D21D0D
:1053A300AE53AF54900006E0FCA3E0FDEFC39DEEC7
:1053B3009C40159000C5E0B40104C2968002C295DA
:1053C3007446900036F0C21DA21DB3B3500790007F
:1053D30036E0B55D0280159000C5E0B40104C296C5
:1053E3008002C2957446900036F0C21D9000C7E05B
:1053F300B40202800302550B900061E0D39565501F
:1054030064900061E0F4042565FE9000CAE08E001C
:10541300F5F0E884FF7E008F72EFC39410500CEF19
:105423008572F0A4FDACF08D7280037572FF90005D
:1054330061E0D39572400B900061E0C39572F57003
:1054430080037570009000E5E0D3957040069000EE
:10545300E5E0F5709000E6E0C3957050069000E635
:10546300E0F5708071900061E0C39565FE9000CA1D
:10547300E08E00F5F0E884FF7E008F72EFC3941096
:10548300500CEF8572F0A4FDACF08D728003757241
:10549300FF85725A755900900061E0255AFFAE5995
:1054A30050010E8E598F5A74FFBE0009D39F4005D9
:1054B300855A7080037570FF9000E5E0D3957040C6
:1054C300069000E5E0F5709000E6E0C395705006A5
:1054D3009000E6E0F570A20DB3B3500D900062E0CA
:1054E300FE9000D2E0D39E5002800A740790003EE3
:1054F300F0C297801375A710E5CDC395704004C221
:10550300978002D29775A700E56EC39409500AA24B
:10551300EDB34005C2ED122C7AAE53AF5474B8C349
:105523009F74889E400C900060E0C3945A4003022D
:10553300577DA215B34009123A69740690003EF0F4
:10554300A220B34008E5B54404F5B58006E5B5549B
:10555300FBF5B5A217B3500EE560D394334007E5CE
:1055630060C394CC4002802FE5B54401F5B57407C0
:1055730090005FF0900073E075F0BEA4FFAEF08E74
:105583005B8F5C7402BE000AD39F4006755C027594
:105593005B00123B3FD217900060E0D394014007B9
:1055A300E560C3941A40028002C2179006B6E06019
:1055B30003122114A22C300301B35017A22CB340C1
:1055C30008E5B54408F5B58006E5B554F7F5B5A289
:1055D3002C92039006BAE060031221F0A22D30044E
:1055E30001B35017A22DB34008E5B54402F5B580C9
:1055F30006E5B554FDF5B5A22D92049006BEE06014
:10560300031222E0A22E300501B3500FA22EB340A5
:1056130004D2A08002C2A0A22E92059006C2E0602E
:10562300031223BCA22F300601B3500FA22FB340A5
:1056330004D2978002C297A22F92069006C6E0601A
:1056430003122498A230300701B3500FA230B340A5
:1056530004D2A28002C2A2A23092079006CAE060DE
:1056630003122574A231300801B3500FA231B340A5
:1056730004D2A18002C2A1A23192089006CEE060BA
:1056830003122650A232300901B35017A232B3409D
:1056930008E5B54440F5B58006E5B554BFF5B5A2B8
:1056A3003292099006D2E0600312272CA233300A0B
:1056B30001B35017A233B34008E5B54480F5B58074
:1056C30006E5B5547FF5B5A233920A9006D6E0609D
:1056D30003122808A234300B01B3500FA234B34095
:1056E30004D2878002C287A234920B9006DAE0606C
:1056F300031228E4A235300C01B3500FA235B34096
:1057030004D2908002C290A235920C900060E0C354
:10571300945A5010E56EB40909900060E004F075E6
:105723006E00803BE56EB40903756E007554007519
:105733005300758D00758B0075630090005FE0C3A7
:10574300940A500890005FE004F08006740A900009
:105753005FF090005FE0B40A06E5B554FEF5B5903E
:105763000060E0D394014007E569C394414002809F
:0D57730009740E90003EF0123A690243598D
:105810000000010001400160018001A001C001E021
:1058200002000300039603B603D603F40400050048
:105830000512052405360548055A056C057E0590B8
:1058400005A805C005DE0600061406280646066EF5
:1058500006AE00FF013F015F017F019F01BF01DF35
:1058600001FF02FF039503B503D503F303FF04FF14
:1058700005110523053505470559056B057D058F80
:1058800005A705BF05DD05F1061306270645066DCC
:1058900006AD06ED0FAA0FA50F9F0F9A0F940F8D5F
:1058A0000F870F800F780F710F680F600F570F4E23
:1058B0000F450F3B0F300F250F1A0F0E0F020EF57D
:1058C0000EE80EDB0ECC0EBE0EAE0E9F0E8E0E7DC3
:1058D0000E6C0E5A0E470E340E200E0C0DF70DE214
:1058E0000DCB0DB50D9D0D850D6D0D540D3A0D2093
:1058F0000D050CE90CCE0CB10C940C760C580C3A3E
:105900000C1B0BFB0BDB0BBB0B9A0B790B570B35F3
:105910000B130AF10ACE0AAB0A870A640A400A1C72
:1059200009F809D409B0098C09670943091F08FB64
:1059300008D608B2088E086A0846082307FF07DC65
:1059400007B9079607730751072F070D06EC06CA1C
:1059500006AA068906690649062A060A05EC05CD47
:1059600005B0059205750558053C0520050504EAB6
:1059700004CF04B5049C0482046904510439042250
:10598000040B03F403DE03C803B2039D038903750C
:105990000361034D033B03280316030402F202E1F3
:1059A00002D102C002B002A002910282027302651B
:1059B00002570249023C022F02220216020901FD8F
:1059C00001F201E601DB01D001C601BB01B101A773
:1059D000019D0194018B01820179017001680160D0
:1059E000015801500148014101390132012B0125C3
:1059F000011E01180111010B010500FF00FA0FA69D
:105A00000FA00F990F920F8B0F840F7C0F740F6BE9
:105A10000F620F580F4E0F430F380F2C0F1F0F122E
:105A20000F050EF70EE80ED80EC80EB70EA50E9392
:105A30000E800E6C0E580E420E2C0E150DFD0DE450
:105A40000DCB0DB10D950D790D5D0D3F0D200D01A7
:105A50000CE10CC00C9E0C7C0C590C350C100BEAA4
:105A60000BC40B9E0B760B4F0B260AFD0AD40AAA19
:105A70000A800A550A2A09FF09D409A8097C095095
:105A8000092508F908CD08A10875084A081E07F37A
:105A900007C8079D07730749072006F706CE06A625
:105AA000067E06570630060A05E405BF059B057706
:105AB00005540532051004EF04CE04AE048F0471C2
:105AC00004530435041903FD03E203C703AD039433
:105AD000037B0363034B0334031E030802F302DE5C
:105AE00002CA02B602A30291027F026D025C024C5E
:105AF000023C022C021D020E020001F201E401D759
:105B000001CA01BE01B101A6019A018F0185017A86
:105B100001700166015D0153014A01410139013102
:105B20000129012101190112010B010400FD00F7F7
:105B300000F000EA00E400DE00D900D300CE00C986
:105B400000C400BF00BA00B500B100AD00A800A4B9
:105B500000A0009C009900950091008E008A0087AB
:085B600000840081007E007B3F
:10009E007547009007B3E4F0A3F07531007530009A
:1000AE00754D00754E00C237D23874FE9007BDF8FC
:1000BE00E4F0E8A3F074FE9007BFF8E4F0E8A3F0D4
:1000CE00745A9007C1F0745A9007C2F0D239C22BFD
:1000DE00C23BC23622750B00750A00AE0AAF0BACDE
:1000EE0008AD09EDC39FEC9E401674FF125F0875B4
:1000FE00CF01780B740126F6500418E436F650DB67
:10010E002290003BE0B4AA1C90076FE0B43C15901F
:10011E0007AFE0FEA3E0FFEF4E6009741EBE0004C1
:10012E00D39F500302023D755C00755B0075F809A4
:10013E009007AFE0FEA3E0FF74076F4E6006740EEB
:10014E006F4E7006743A90076FF09007AFE0FEA303
:10015E00E0FF7408BE001ED39F401A7E017F0890F8
:10016E0007AFE0FCA3E0FD1DBDFF011C1200038ED6
:10017E00598F5A801F9007AFE0FEA3E0FF7408125C
:10018E005F6C8F048E057E017F08CDCCCD120003EF
:10019E008E598F5AAE5BAF5C740CD39F74019E5018
:1001AE0003020238A2F9B3407EE55C455B7003752D
:1001BE00A382AE5BAF5C74016F4E700375A300AE8D
:1001CE005BAF5C74026F4E700D9007B0E075F0027D
:1001DE00A4FDACF08DA3AE5BAF5C74036F4E7003E9
:1001EE0075A300AE5BAF5C7403BE00039F5013ACEF
:1001FE0059AD5AED2FFFEC3EFE90006B125F4FE0B3
:10020E00F5A3AE5BAF5CEFB40B09EEB4010574144D
:10021E00125F08AE5BAF5CEFB40B07EEB401037573
:10022E00F80D785B125F7C0201A290003BE4F02295
:10023E00755C00755B0075F8099007AFE0FEA3E0F2
:10024E00FF7408BE001ED39F401A7E017F089007E0
:10025E00AFE0FCA3E0FD1DBDFF011C1200038E5993
:10026E008F5A801F9007AFE0FEA3E0FF7408125F65
:10027E006C8F048E057E017F08CDCCCD1200038ECF
:10028E00598F5AAE5BAF5C7411D39F74019E5003AD
:10029E0002036EA2F9B3500302036BE55C455B707B
:1002AE000375A3D2AE5BAF5C74016F4E700375A382
:1002BE0000AE5BAF5C74026F4E700D9007B0E075D0
:1002CE00F002A4FDACF08DA3AE5BAF5C74036F4E79
:1002DE00700375A300AE5BAF5C74046F4E70037554
:1002EE00A300AE5BAF5C74056F4E700375A300AEDA
:1002FE005BAF5C74066F4E700375A300AE5BAF5CB4
:10030E0074076F4E700375A300AE5BAF5C74086F1D
:10031E004E700375A300AE5BAF5C7408BE00039F06
:10032E005016AC59AD5AED2FFFEC3EFE9000661202
:10033E005F4FE5A3F075A300AE5BAF5CEFB41009A1
:10034E00EEB401057414125F08AE5BAF5CEFB4102F
:10035E0007EEB4010375F80D785B125F7C02029113
:10036E0022755C00755B0075F809AE5BAF5C7417A7
:10037E00BE0004D39F5003020447A2F9B3500302F8
:10038E000444E55C455B700375A3D2AE5BAF5C7451
:10039E00016F4E700375A300AE5BAF5C74026F4EBF
:1003AE00700D9007B0E075F002A4FDACF08DA3AE19
:1003BE005BAF5C74036F4E700375A300AE5BAF5CF6
:1003CE0074046F4E700375A300AE5BAF5C74056F63
:1003DE004E700375A300AE5BAF5C74066F4E700378
:1003EE0075A300AE5BAF5C74076F4E700375A30010
:1003FE00AE5BAF5C74086F4E700375A300AE5BAF5F
:10040E005C7408BE00039F500C900048125F4FE5CD
:10041E00A3F075A300AE5BAF5C74166F4E700574DF
:10042E0014125F08AE5BAF5C74166F4E700375F8F6
:10043E000D785B125F7C0203782290003BE0B4AB38
:10044E000280030204E2755C00755B0075F809AE6C
:10045E005BAF5C7412BE007CD39F4078A2F9B340B0
:10046E0070E55C455B700375A382AE5BAF5C740197
:10047E006F4E700375A300AE5BAF5C74026F4E706F
:10048E000D9007B0E075F002A4FDACF08DA3AE5B4D
:10049E00AF5C74036F4E700375A300AE5BAF5C74FC
:1004AE0003BE00039F500990004D125F4FE0F5A36D
:1004BE00AE5BAF5C74116F4E70057414125F08AEB4
:1004CE005BAF5C74116F4E700375F80D785B125F45
:1004DE007C02045D229007BAE4F074649007AFF8D2
:1004EE00E4F0E8A3F012036F74C89007AFF8E4F0DD
:1004FE00E8A3F0900054E0B4371A900051E0900059
:10050E0048F0900052E0900049F0900053E09000C7
:10051E004AF080469007BA7401F074659007AFF800
:10052E00E4F0E8A3F012036F74C89007AFF8E4F09C
:10053E00E8A3F0900054E0B4371A900051E0900018
:10054E0048F0900052E0900049F0900053E0900087
:10055E004AF0800674029007BAF09007BBE4F0747C
:10056E00669007AFF8E4F0E8A3F012036F74C8903A
:10057E0007AFF8E4F0E8A3F0900053E0B437129020
:10058E000051E0900042F0900052E090004BF0805D
:10059E00769007BB7401F074679007AFF8E4F0E84B
:1005AE00A3F012036F74C89007AFF8E4F0E8A3F05D
:1005BE00900053E0B43712900051E0900042F0905A
:1005CE000052E090004BF0803E74029007BBF07436
:1005DE00689007AFF8E4F0E8A3F012036F74C890C8
:1005EE0007AFF8E4F0E8A3F0900053E0B4371290B0
:1005FE000051E0900042F0900052E090004BF080ED
:10060E000674039007BBF022E54E64046006E5997C
:10061E0064FF6002802AA2374004D2378020E54E64
:10062E00600874E6254E90003EF0754E00E54D6074
:10063E000874F0254D90003EF0754D00C2378002D3
:10064E00C237E54E9033F8F8282873754E00E599B9
:10065E00B4FF03754D01E599B4FE03754D02E5999E
:10066E00B4FD03754D03E599B4FC03754D04E5998E
:10067E00B4FA03754D05E599B4FB06754E01123AB1
:10068E0069E599B4F906754E04123A69E599D39461
:10069E00E54007E599C394F04002801685994F75A1
:1006AE004E027E017F00E54FC394E6125F288E3224
:1006BE008F339007B3E4F0A3F0E599D394C44007C9
:1006CE00E599C394E64002802885994F754E0374D0
:1006DE00E5C3954FF533753200AE32AF33905810F7
:1006EE00125EF7E493F87401939007B3C8F0A3C8B1
:1006FE00F0D299020AB3900051E070429007B3E035
:10070E00FEA3E0FF74FFBE00039F5009EFC39446A3
:10071E00EE940640119007B3E0FEA3E0FFEFD394F2
:10072E006DEE940640139007B3E0FEA3E0FF900039
:10073E006F125F4FE599F0800385997380119007D2
:10074E00B3E0FEA3E0FF90006F125F4FE599F090CB
:10075E0007B3125F369007B3E0FEA3E0FFEFB401DC
:10076E0006EEB40702800302089B90076FE0B43CCC
:10077E00028003020885C29C900051E090010DF0AA
:10078E00900052E090007CF0900053E090009CF0BE
:10079E00900054E09000C5F0900055E0900071F08C
:1007AE00900056E09000B7F0900057E09000D5F022
:1007BE00900058E09000A9F0900059E09000C7F02A
:1007CE0090005AE09000F7F01236F0900063E0903F
:1007DE0000DEF0900064E0900095F0900065E090EF
:1007EE000096F074639007AFF8E4F0E8A3F074ABF2
:1007FE0090003BF012044890003BE4F075096475DC
:10080E0008001200E3A21F4038757201E572D394FE
:10081E0007502CE5729007AFF8E4F0E8A3F074AA45
:10082E0090003BF012010FE572C394075009750951
:10083E00647508001200E37872740126F650CD80BC
:10084E0036757208E572D3940E502CE5729007AF90
:10085E00F8E4F0E8A3F074AA90003BF012010FE563
:10086E0072C3940E50097509647508001200E3787E
:10087E0072740126F650CD74C89007AFF8E4F0E814
:10088E00A3F0D29C754E00754D007599FB020AB30C
:10089E009007B3E0FEA3E0FFEF4E70068599317529
:1008AE0030009007B3E0FEA3E0FF74016F4E701BA3
:1008BE00AC30AD31AA32AB33ED2BFBEC3AFA8A06F3
:1008CE008B0790006F125F4FE599F09007B3125FA0
:1008DE00369007B3E0FEA3E0FF74026F4E7021ACBA
:1008EE0030AD3174566D4C7006E54F64E660028093
:1008FE0003123A691236F0854F99754E00754D0008
:10090E00020AB39007B3E0FEA3E0FF90006F125F00
:10091E004FE599F09007B3125F369007B3E0FEA350
:10092E00E0FFAC32AD338F028E038C068D079058EC
:10093E0052125EF7E493F9740193FEEAD39EEB999B
:10094E004009854F99754E00754D00020AB3900708
:10095E00B3E0FEA3E0FF90006F125F4FE599F090B9
:10096E0007B3125F369007B3E0FEA3E0FFEFB400CB
:10097E0006EEB401028003020AB390004AE075F05D
:10098E0002A4FDACF08D72ED90006F125F5AEDFA7D
:10099E00E0FBEA900072125F5AEBFAE0FBEA2BFAE8
:1009AE0090004AE0B502028003020AA50DED900008
:1009BE006F125F5AE572FDE0FAED900073125F5A06
:1009CE00EAFDE0FAEDC39AFD90004AE0B50502801B
:1009DE0003020AA5E572900071125F5AE572FDE0FE
:1009EE00FAED900074125F5AEAFDE0FAED2AFD90DE
:1009FE00004AE0B505028003020AA5E57290007573
:100A0E00125F5AFDE0FAED90004AE0F4042A9000DD
:100A1E0051F0E572900076125F5AFDE0FAED90000B
:100A2E004AE0F4042A900052F0E572900077125FCB
:100A3E005AFDE0FAED90004AE0F4042A900053F0DB
:100A4E00E572900078125F5AFDE0FAED90004AE0F0
:100A5E00F4042A9007AFF8E4F0E8A3F074AB90002A
:100A6E003BF01204487509647508001200E3900704
:100A7E00AF125F361204487509647508001200E360
:100A8E009007AF125F361204487599F975096475AF
:100A9E0008001200E380FE7599FF75096475080061
:050AAE001200E380FED0
:0F33F80002065902070402089E02091102095C2D
:100AB30022E54D903407F8282873020B989007B36A
:100AC300E0FEA3E0FF900040125F4FE0F59990072E
:100AD300B3125F369007B3E0FEA3E0FF74116F4ECD
:100AE3007003754D00020B98856D99020B98900762
:100AF300B3E0FEA3E0FF90006F125F4FE0F599EFC4
:100B0300B40107EEB40703754D009007B3125F36C7
:070B1300020B989007B4E00B
:0F340700020ABD020AC0020AEB020AF1020B160A
:100B1A009035BAF82828738552998067855E99803E
:100B2A0062856099805D856499805885669980534D
:100B3A00856799804E85689980498569998044902E
:100B4A000016E0F599803CA238B340077599FAC2BD
:100B5A00388017A229B3400575990F800B90003E83
:100B6A00E0F59990003EE4F0C2298017856A9980E1
:100B7A0012856599800D856B9980087599FC8003AB
:030B8A00754D00A6
:1035BA00020B21020B26020B2B020B30020B3502E7
:1035CA000B3A020B3F020B44020B49020B51020B4E
:0D35DA0076020B7B020B80020B85020B8A30
:0B0B8D009007B3125F3680031235E7BB
:03341600020B9511
:100B980022E537255AFFAE5950010E90006F125FBB
:100BA8004FE0F538E537255AFFAE5950010E0FBF13
:100BB80000010E90006F125F4FE0F539853F3BE56D
:100BC80038B539058538378041E539D39538401D22
:100BD800E539C39538853AF0A4FFAEF0E53B8E04BD
:100BE8008F05FF125F18ED2538F537801DE538C3EE
:100BF8009539853AF0A4FFAEF0E53B8E048F05FFEA
:100C0800125F18EDF4042538F53722E539D3953805
:100C1800401DE539C39538853AF0A4FFAEF0E53BB1
:100C28008E048F05FF125F18ED2538F537801DE516
:100C380038C39539853AF0A4FFAEF0E53B8E048FB2
:100C480005FF125F18EDF4042538F537229000757A
:100C5800E0B40170E56675F00A84FF7E008F37E521
:100C68006675F00A84ADF07C008D3A753F0A7559B7
:100C780005755A24E537C394115005120B9980065F
:100C88009005A4E0F537E537900068F0E56675F063
:100C98000A84FF7E008F37E56675F00A84ADF07C24
:100CA800008D3A753F0A755905755A5AE537C39448
:100CB800115005120B9980069005DAE0F537E537F3
:100CC80090000EF022900075E0B4016AE56675F0B8
:100CD8000A84FF7E008F37E56675F00A84ADF07CE4
:100CE800008D3A753F0A755905755A36E537C3942C
:100CF800115005120B9980069005B6E0F537853737
:100D08004BE56675F00A84FF7E008F37E56675F05F
:100D18000A84ADF07C008D3A753F0A755905755AFD
:100D280048E537C394115005120B9980069005C801
:100D3800E0F53785374C22E55E75F00484FF7E00C8
:100D48008F37E55E75F00484ADF07C008D3A753F11
:100D580004755901755A00E537C3943F5005120BC5
:100D68009980069001AEE0F53785372975280090FF
:100D7800003DE075F020A4FFAEF09000C0E08E04C6
:100D88008F05FF125F188D379000A8E0D3955E504D
:100D980003020E459000CCE0D3955E4010ED900123
:100DA800AF125F5AE0F52B752A00020E42900097A9
:100DB800E0D3955E4043E5379001AF125F5AE0F506
:100DC80038E5379001CF125F5AE0F5399000CCE052
:100DD800F404255EF53A900097E0FE9000CCE0F42C
:100DE800042EF53BE538B539058538378003120CF4
:100DF8001385372B752A008041E5379001CF125FA4
:100E08005AE0F538E5379001EF125F5AE0F539906E
:100E18000097E0F404255EF53A9000A8E0FE900003
:100E280097E0F4042EF53BE538B539058538378069
:100E380003120C1385372B752A00020EEC9000CF95
:100E4800E0D3955E5011E53790022F125F5AE0F516
:100E58002B752A00020EEC900098E0D3955E504363
:100E6800E53790020F125F5AE0F538E53790022F08
:100E7800125F5AE0F539900098E0F404255EF53ADF
:100E88009000CFE0FE900098E0F4042EF53BE538A2
:100E9800B539058538378003120C1385372B752A29
:100EA800008041E5379001EF125F5AE0F538E537E9
:100EB80090020F125F5AE0F5399000A8E0F404257B
:100EC8005EF53A900098E0FE9000A8E0F4042EF554
:100ED8003BE538B539058538378003120C1385375B
:100EE8002B752A00229000E0E0F53C753F117559FA
:100EF80002755A00AE51AF52E53C75F00FA4FDAC37
:100F0800F0EDD39FEC9E4021E53C8E048F05FF1247
:100F18005F18ED75F010A4FFAEF0E55E75F0118472
:100F2800FD7C00ED2FF53D800EE55E75F01184FF28
:100F38007E00EF24F0F53D853D37E55E75F01184C0
:100F4800AFF07E008F3A120B9985373EAE51AF5203
:100F58009000E0E075F00FA4FDACF0EDD39FEC9E9F
:100F68004028755902755A10853D37120B99853EF0
:100F780038853739AE51AF52E53C8E048F05FF12E4
:100F88005F438D3A853C3B120C1385372975280041
:100F9800752B64752A00229000E0E0F53C753F113E
:100FA800755902755A00AE51AF52E53C75F00FA461
:100FB800FDACF0EDD39FEC9E4021E53C8E048F05FF
:100FC800FF125F18ED75F010A4FFAEF0E56075F044
:100FD8001184FD7C00ED2FF53D800EE56075F01164
:100FE80084FF7E00EF24F0F53D853D37E56075F020
:100FF8001184AFF07E008F3A120B9985373EAE51BF
:10100800AF529000E0E075F00FA4FDACF0EDD39F77
:10101800EC9E4028755902755A10853D37120B9978
:10102800853E38853739AE51AF52E53C8E048F0581
:10103800FF125F438D3A853C3B120C1385372975A7
:1010480028009000AAE0B40453E55E75F00484FF1C
:101058007E008F37E55E75F00484ADF07C008D3A34
:10106800753F04755901755A00E537C3943F50051B
:10107800120B9980069001AEE0F537AE28AF29E54E
:1010880037125F2874648E048F05FF125F18AE282C
:10109800AF29EF2DFDEE3CFC8C288D29752B64754E
:1010A8002A0022900075E0B40146E56675F00A84CE
:1010B800FF7E008F37E56675F00A84ADF07C008D01
:1010C8003A753F0A755905755A00E537C3941150AA
:1010D80005120B998006900580E0F537AE2AAF2BF4
:1010E800E5372FFF50010E7464125F6C8E2A8F2B28
:1010F800900076E0B40146E56775F00A84FF7E004B
:101108008F37E56775F00A84ADF07C008D3A753F3E
:101118000A755905755A6CE537C394115005120BB9
:101128009980069005ECE0F537AE2AAF2BE5372F0E
:10113800FF50010E7464125F6C8E2A8F2B9000850D
:10114800E0B40249E569C3944175F00584FF7E0067
:101158008F37E56975F00584ADF07C008D3A753FF1
:1011680005755906755A00E537C394135005120BD7
:10117800998006900682E0F537AE2AAF2BE5372F27
:10118800FF50010E7464125F6C8E2A8F2B9000C77B
:10119800E0B40202800302124AE55E75F01584FF8E
:1011A8007E008F37E55E75F01584ADF07C008D3AD2
:1011B800753F15755903755AF4E537C3940B5005F7
:1011C800120B99800690046EE0F537E53775F0FF4D
:1011D800A4FFAEF09000C8E08E048F05FF125F18E0
:1011E800ED900061F0E56575F078A4FFAEF074FF4E
:1011F8008E048F05FF125F188C598D5A74028C0665
:101208008D071200398F37AC59AD5A7404FF125F3D
:10121800438D3A753F04755906755A28E537C394C6
:101228001D5005120B9980069006B4E0F537AE2ADA
:10123800AF2BE5372FFF50010E7464125F6C8E2AB6
:101248008F2B900074E0B4025DE56075F064A4FF34
:10125800AEF074081200398E5B8F5C74058E048FB3
:1012680005FF125F188D37AE5BAF5C74058E048F77
:1012780005FF125F438D3A753F05755905755ADEAE
:10128800E537C394135005120B998006900660E069
:10129800F537AE2AAF2BE5372FFF50010E746412D5
:1012A8005F6C8E2A8F2B9000B6E0703C90003DE07A
:1012B80075F00584FF7E008F3790003DE075F005DE
:1012C80084ADF07C008D3A753F05755905755AC097
:1012D800E537C3941D5005120B99800690064CE023
:1012E800F537E537900069F02290007DE0B40117EA
:1012F8009007B6E0252BFFAE2A50010E9000D1E0F2
:10130800125F6C8E2A8F2B9000F5E0B401149000C8
:10131800F6E0A851B8000495525007E55EC3955F02
:101328004002801290009FE0252BFFAE2A50010E4C
:101338008E2A8F2B802F90007DE0B40316A22BB34A
:10134800B350109007B9E0C39405A851B8000695AA
:10135800524002801090009FE0252BFFAE2A5001DA
:101368000E8E2A8F2B900077E0B4020280030215BC
:101378004D90007AE0602FE566D3944640289000AF
:101388000FE0FEA3E0FF9000B5E075F003A4FDAC0C
:10139800F0EFD39DEE9C400E9000D9E0A851B80024
:1013A80005D39552500302154D9000C2E0855EF0BA
:1013B800A4FFAEF07405125F2874071200398E5925
:1013C8008F5A900081E0A851B800049552501290AD
:1013D8000082E075F002A4FDACF0EFC39DEE9C40E6
:1013E8000302154DE55E75F00B84FF7E009005FF46
:1013F800125F4FFEE0FFEE900079E0FEEF8E00886E
:10140800F0A4FFAEF074648E048F05FF125F188C91
:10141800598D5A90003DE075F018A4FFAEF0900089
:10142800C0E08E048F05FF125F188C068D079006AA
:1014380017125F4FAE59AF5AE0125F2874648E04DA
:101448008F05FF125F188C598D5AE564A859B800AA
:1014580077D3955A4072E564C3955AFFE49559FECF
:101468008E598F5A7428BE00039F500C755A2875E0
:101478005900740D90003EF0AE59AF5A90007AE0D2
:10148800125F2874288E048F05FF125F188C598DFF
:101498005AAE28AF29740A8E048F05FF125F188D83
:1014A800068C07AC59AD5ACFCECF120003740A8E02
:1014B800048F05FF125F188C598D5AAE28AF291278
:1014C8005F748E288F29807DE564A859B80004953B
:1014D8005A5072AE59AF5AE564125F6C8E598F5AE2
:1014E8007428BE00039F500C755A28755900740D56
:1014F80090003EF0AE59AF5A90007AE0125F28741F
:10150800288E048F05FF125F188C598D5AAE28AFAC
:1015180029740A8E048F05FF125F188D068C07AC9C
:1015280059AD5ACFCECF120003740A8E048F05FF2F
:10153800125F188C598D5AAE28AF29EF2DFDEE3C5D
:10154800FC8C288D29229000D5E0B4026AE55E75EE
:10155800F00884FF7E008F37E55E75F00884ADF0F3
:101568007C008D3A753F08755901755AE0E537C317
:10157800943F5005120B99800690026EE0F537856E
:10158800372D752C00AE2CAF2DAC2AAD2B120003D5
:1015980074648E048F05FF125F188C2C8D2D9000BB
:1015A80072E08C068D07125F2874648E048F05FF25
:1015B800125F188C2C8D2DAE28AF29AC2AAD2B12BA
:1015C800000374648E048F05FF125F188C288D2920
:1015D800900072E08C068D07125F2874648E048F69
:1015E80005FF125F188C288D29A20D401DAE51AF42
:1015F800527405BE00039F5002D20DE560D394CC0F
:101608004008D201741190003EF09000D4E0B4027A
:10161800089000D6E0640160028035AE28AF29E565
:101628006A125F2874E78E048F05FF125F188C28F2
:101638008D299000D5E0B40217AE2CAF2DE56A12C3
:101648005F2874E78E048F05FF125F188C2C8D2D90
:10165800900094E05402601B90008BE0A851B80001
:1016680012D39552400DA20DB3B35007E560C39451
:101678009A40028028AE35AF36900089E075F002B6
:10168800A4FDACF0EF2DFDEE3CFC74022DFD5001E5
:101698000CE560BC0007D39D4003754301856036A7
:1016A800753500E54370030217919000E7E0C39594
:1016B8004350030217839000F7E0C394025076E585
:1016C8006675F00A84FF7E0090056F125F4FE0F5A3
:1016D8005A755900AE59AF5A90008AE0125F2874C3
:1016E800648E048F05FF125F188C5B8D5C9000E799
:1016F800E004C395438C068D07125F289000E7E04D
:101708008E048F05FF125F188C5B8D5CAE28AF29A5
:10171800EF2DFDEE3CFC8C288D299000D5E0B4021D
:1017280012AE2CAF2DAA5BAB5CEF2BFBEE3AFA8A1C
:101738002C8B2D80469000E7E004C39543854BF041
:10174800A4FFAEF09000E7E08E048F05FF125F184B
:101758008C5B8D5CAE28AF29EF2DFDEE3CFC8C2810
:101768008D299000D5E0B40212AE2CAF2DAA5BAB48
:101778005CEF2BFBEE3AFA8A2C8B2D05439000E7A1
:10178800E0C395435003754300900094E054016012
:101798001B900088E0A851B80012D39552400DA2C2
:1017A8000DB3B35007E55EC394CC4002802590008A
:1017B80086E075F003A4FFAEF0E5402FFF50010E60
:1017C80074032FFF50010EE55EBE0007D39F400350
:1017D800754401855E40E54470030218C49000E832
:1017E800E0C3954450030218B69000F7E0C3940292
:1017F8005076E56675F00A84FF7E0090056F125FEB
:101808004FE0F55A755900AE59AF5A900087E0126B
:101818005F2874648E048F05FF125F188C5B8D5CE3
:101828009000E8E004C395448C068D07125F289069
:1018380000E8E08E048F05FF125F188C5B8D5CAEAC
:1018480028AF29EF2DFDEE3CFC8C288D299000D582
:10185800E0B40212AE2CAF2DAA5BAB5CEF2BFBEE13
:101868003AFA8A2C8B2D80469000E8E004C3954410
:10187800854CF0A4FFAEF09000E8E08E048F05FFE1
:10188800125F188C5B8D5CAE28AF29EF2DFDEE3C06
:10189800FC8C288D299000D5E0B40212AE2CAF2D17
:1018A800AA5BAB5CEF2BFBEE3AFA8A2C8B2D054436
:1018B8009000E8E0C3954450037544009000EAE0C6
:1018C8002529FFAE2850010E8E288F29900099E017
:1018D800A828B8000495295009900099E0F52975C1
:1018E80028009000D5E0B4020D900099E0A82CB82B
:1018F8000006952D40028009900099E0F52D752C81
:1019080000229000D5E0B401028003021A15A20D4E
:10191800B35003021A139000A0E0B40168AE28AFD8
:1019280029AC51AD52120003743C8E048F05FF128E
:101938005F189000B0E0BC00109D400D9000B2E030
:10194800A828B8000495295002D202AE28AF29ACC5
:1019580051AD52120003743C8E048F05FF125F18BC
:101968009000B0E0C3940ABC0015D39D40119000CC
:10197800B2E0C39405A828B80005D3952950028081
:1019880002C2028068AE28AF29AC51AD52120003E2
:1019980074788E048F05FF125F189000B0E0BC00C9
:1019A800109D400D9000B2E0A828B8000495295079
:1019B80004D2028038AE28AF29AC51AD52120003D0
:1019C80074788E048F05FF125F189000B0E0C394FE
:1019D8000ABC0015D39D40119000B2E0C39405A83D
:1019E80028B80005D3952950028002C202A202B38A
:1019F8004019AE28AF299000B1E0125F2874648EB8
:101A0800048F05FF125F188C288D298002C202A25C
:101A180000B34006A201B3B35009900015E4F0A347
:101A2800F08024AE28AF297400D39F74019E400C27
:101A3800900015E528F0A3E529F0800B74FF9000CD
:101A480015F8E4F0E8A3F09000B7E0D39402400C56
:101A58009000A2E07006A20DB3B34002801AAE282F
:101A6800AF297402125F288E288F29AE2CAF2D74EF
:101A780002125F288E2C8F2D9000A0E0B4011AAEC0
:101A880028AF297402125F288E288F29AE2CAF2D1B
:101A98007402125F288E2C8F2DAE28AF29745E1227
:101AA8005F28740A8E048F05FF125F188C288D2911
:101AB8009000D5E0B40217AE2CAF2D745E125F28EB
:101AC800740A8E048F05FF125F188C2C8D2DAE289A
:101AD800AF297402BE000AD39F40067529027528F3
:101AE80000AE2CAF2D7402BE000AD39F4006752DA0
:101AF80002752C00900013E528F0A3E529F0229048
:101B0800003DE090036F125F5AE0F5417542649022
:101B1800003DE0FE9000ABE0D39E4037E55E75F0F7
:101B28000884FF7E008F37E55E75F00884ADF07C91
:101B3800008D3A753F08755903755A96E537C39471
:101B48001F5005120B998006900424E0F53785375D
:101B5800428035E55E75F00884FF7E008F37E55ECC
:101B680075F00884ADF07C008D3A753F087559030F
:101B7800755AB6E537C3941F5005120B9980069025
:101B88000444E0F537853742229000E1E0F53C75E2
:101B98003F11755904755A00AE51AF52E53C75F0C6
:101BA8000FA4FDACF0EDD39FEC9E4021E53C8E04E4
:101BB8008F05FF125F18ED75F010A4FFAEF0E55E1B
:101BC80075F01184FD7C00ED2FF53D800EE55E7506
:101BD800F01184FF7E00EF24F0F53D853D37E55E8A
:101BE80075F01184AFF07E008F3A120B9985373E5D
:101BF800AE51AF529000E1E075F00FA4FDACF0EDEE
:101C0800D39FEC9E4028755904755A10853D3712AC
:101C18000B99853E38853739AE51AF52E53C8E0475
:101C28008F05FF125F438D3A853C3B120C138537B5
:101C380041754264229000E1E0F53C753F11755909
:101C480004755A00AE51AF52E53C75F00FA4FDACD7
:101C5800F0EDD39FEC9E4021E53C8E048F05FF12EA
:101C68005F18ED75F010A4FFAEF0E56075F0118413
:101C7800FD7C00ED2FF53D800EE56075F01184FFC9
:101C88007E00EF24F0F53D853D37E56075F0118461
:101C9800AFF07E008F3A120B9985373EAE51AF52A6
:101CA8009000E1E075F00FA4FDACF0EDD39FEC9E41
:101CB8004028755904755A10853D37120B99853E91
:101CC80038853739AE51AF52E53C8E048F05FF1287
:101CD8005F438D3A853C3B120C138537417542644E
:101CE8009000DCE0B4047990003DE0FE9000ABE0A9
:101CF800D39E4037E55E75F00884FF7E008F37E598
:101D08005E75F00884ADF07C008D3A753F08755912
:101D180003755A96E537C3941F5005120B99800630
:101D2800900424E0F5378537428035E55E75F00884
:101D380084FF7E008F37E55E75F00884ADF07C0087
:101D48008D3A753F08755903755AB6E537C3941F20
:101D58005005120B998006900444E0F53785374208
:101D680022900075E0B4013BE56675F00A84FF7EB9
:101D7800008F37E56675F00A84ADF07C008D3A7502
:101D88003F0A755905755A12E537C3941150051263
:101D98000B998006900592E0F537E5422537C39404
:101DA80064F542900076E0B4013BE56775F00A847B
:101DB800FF7E008F37E56775F00A84ADF07C008DF3
:101DC8003A753F0A755905755A7EE537C39411501F
:101DD80005120B9980069005FEE0F537E542253798
:101DE800C39464F542E5412542F53490007DE0B4A2
:101DF80002109007B5E02534FE9000D1E0F4042EDF
:101E0800F5349000D4E0D394014040E56AC394E7E8
:101E1800501D74E7C3956AFE9007B7E08E00F5F091
:101E2800E884FF7E008F37E5342537F534801CE5DC
:101E38006AC394E7FE9007B7E08E00F5F0E884FFE8
:101E48007E008F37E534C39537F534A20D4006E59B
:101E5800412464F534E534D394644009E534C394EB
:101E680064F53480037534009000ADE0C3953450B8
:101E7800069000ADE0F53422D200900067E0A8514A
:101E8800B8000495525041900067E0A851B800048A
:101E98009552500375340F900067E004A851B800BC
:101EA800049552500375340A900067E02402A85143
:101EB800B8000495525005753405C200900067E0DB
:101EC8006006740990003EF0C23B7E017F009000DE
:101ED800B3E0125F289000C2E08E048F05FF125F06
:101EE80018E55EBC0017D39D40139000BCE0B40217
:101EF80004D23B8002C200740A90003EF09000B405
:101F0800E0C3956650159000C6E0A851B800049546
:101F1800525002C200740B90003EF0E566C3946410
:101F2800501D90010CE0600D90010CE0A851B80024
:101F380006955240028008C200740B90003EF0A241
:101F48000040037534059000F5E0B401149000F6E4
:101F5800E0A851B8000495525007E55EC3955F406C
:101F680002800890009EE0F534803A90007DE0B44D
:101F78000306A22BB3B34002802B9007B9E0C394A9
:101F880005A851B800049552500C90009EE0F53415
:101F9800740C90003EF09007B9E0A851B800049581
:101FA800525002C20085346B90006FE02534FE90D9
:101FB800003DE075F01E84FC7F00EE2CF534229085
:101FC800003DE075F00584FF7E008F3790003DE00E
:101FD80075F00584ADF07C008D3A753F05755903A1
:101FE800755AD69000C0E01475F00584FF7E00E5B0
:101FF80037BE00039F5005120B99800BE5379004FC
:1020080045125F5AE0F537E5379007B8F09007B802
:10201800E0FE9000AFE0C39E50089000AFE090074C
:10202800B8F022E56675F00A84FF7E0090056F120D
:102038005F4FE0F546E546D394644010E546C39407
:102048006475F00F84FF7E008F468003754600900C
:102058000092E02546F546229007A9E0FEA3E0FF9E
:102068007404120039E55E125F28740F8E048F0520
:10207800FF125F189007A7ECF0A3EDF0900085E041
:10208800B40262E569C3944175F00584FF7E008F50
:1020980037E56975F00584ADF07C008D3A753F052C
:1020A800755906755A14E537C394175005120B99DC
:1020B8008006900696E0F5379007A7E0FEA3E0FFBC
:1020C800740A8E048F05FF125F18E5378C068D079A
:1020D800125F28740A8E048F05FF125F189007A7F5
:1020E800ECF0A3EDF09007A7E0FEA3E0FF9007ADAA
:1020F800E0FCA3E0FDEDD39FEC9E400F9007ADE020
:10210800F8A3E09007A7C8F0A3C8F0229006B6E0AD
:10211800903419F8282873804C85527280479000B3
:10212800C2E0855EF0A4FFAEF074081200398F7229
:102138008033856072802E856672802985677280FB
:1021480024856872801F856972801A856A72801575
:102158008565728010856472800B856B728006902D
:052168000016E0F57215
:1034190002211F02212102212602213A02213F0213
:10342900214402214902214E02215302215802213D
:073439005D02216202216720
:10216D009006B7E0FE9006B8E0D39E404B9006B6C1
:10217D00E0B404189006B8E0C395725002D22C90CA
:10218D0006B7E0D395724002C22C802A9006B7E0C4
:10219D00C3957250099006B8E0D395725002800233
:1021AD00D22C9006B7E0D3957250099006B8E0C3D3
:1021BD0095725002C22C802A9006B7E0D3957240DA
:1021CD00099006B8E0C3957240028002C22C9006B9
:1021DD00B7E0C3957240099006B8E0D395724002FE
:1021ED00D22C229006BAE0903440F8282873804C07
:1021FD0085527280479000C2E0855EF0A4FFAEF07C
:10220D0074081200398F728033856072802E856656
:10221D007280298567728024856872801F85697236
:10222D00801A856A7280158565728010856472804A
:0C223D000B856B728006900016E0F572B5
:103440000221FB0221FD02220202221602221B029D
:10345000222002222502222A02222F0222340222C4
:073460003902223E02224363
:102249009006BBE0FE9006BCE0D39E405F9006BAC4
:10225900E0B404189006BCE0C395725002D22D90E8
:1022690006BBE0D395724002C22D803E9006BBE0CA
:10227900C3957250099006BCE0D395725002800252
:10228900D22D9006BBE0D3957250099006BCE0C3ED
:1022990095725002C22D9006BAE0B401099000CEA1
:1022A900E0D3956050028002C22D802A9006BBE0DF
:1022B900D3957240099006BCE0C395724002800232
:1022C900C22D9006BBE0C3957240099006BCE0D3CD
:1022D90095724002D22D229006BEE0903467F8280C
:1022E9002873804C85527280479000C2E0855EF069
:1022F900A4FFAEF074081200398F728033856072C2
:10230900802E85667280298567728024856872802F
:102319001F856972801A856A7280158565728010B9
:10232900856472800B856B728006900016E0F572E9
:103467000222EB0222ED0222F202230602230B02C2
:10347700231002231502231A02231F0223240223E7
:073487002902232E0223336A
:102339009006BFE0FE9006C0E0D39E404B9006BEDB
:10234900E0B404189006C0E0C395725002D22E90F2
:1023590006BFE0D395724002C22E802A9006BFE0E4
:10236900C3957250099006C0E0D39572500280025D
:10237900D22E9006BFE0D3957250099006C0E0C3F3
:1023890095725002C22E802A9006BFE0D395724002
:10239900099006C0E0C3957240028002C22E9006E1
:1023A900BFE0C3957240099006C0E0D39572400220
:1023B900D22E229006C2E090348EF8282873804CE1
:1023C90085527280479000C2E0855EF0A4FFAEF0AE
:1023D90074081200398F728033856072802E856689
:1023E9007280298567728024856872801F85697269
:1023F900801A856A7280158565728010856472807D
:0C2409000B856B728006900016E0F572E7
:10348E000223C70223C90223CE0223E20223E7024C
:10349E0023EC0223F10223F60223FB022400022472
:0734AE000502240A02240FAD
:102415009006C3E0FE9006C4E0D39E404B9006C2F2
:10242500E0B404189006C4E0C395725002D22F9010
:1024350006C3E0D395724002C22F802A9006C3E0FE
:10244500C3957250099006C4E0D39572500280027C
:10245500D22F9006C3E0D3957250099006C4E0C30D
:1024650095725002C22F802A9006C3E0D395724020
:10247500099006C4E0C3957240028002C22F9006FF
:10248500C3E0C3957240099006C4E0D3957240023B
:10249500D22F229006C6E09034B5F8282873804CD8
:1024A50085527280479000C2E0855EF0A4FFAEF0D1
:1024B50074081200398F728033856072802E8566AC
:1024C5007280298567728024856872801F8569728C
:1024D500801A856A728015856572801085647280A0
:0C24E5000B856B728006900016E0F5720B
:1034B5000224A30224A50224AA0224BE0224C302D4
:1034C50024C80224CD0224D20224D70224DC0224FB
:0734D500E10224E60224EBF2
:1024F1009006C7E0FE9006C8E0D39E404B9006C60A
:10250100E0B404189006C8E0C395725002D230902E
:1025110006C7E0D395724002C230802A9006C7E018
:10252100C3957250099006C8E0D39572500280029B
:10253100D2309006C7E0D3957250099006C8E0C327
:1025410095725002C230802A9006C7E0D39572403E
:10255100099006C8E0C3957240028002C23090061D
:10256100C7E0C3957240099006C8E0D39572400256
:10257100D230229006CAE09034DCF8282873804CCF
:1025810085527280479000C2E0855EF0A4FFAEF0F4
:1025910074081200398F728033856072802E8566CF
:1025A1007280298567728024856872801F856972AF
:1025B100801A856A728015856572801085647280C3
:0C25C1000B856B728006900016E0F5722E
:1034DC0002257F02258102258602259A02259F025C
:1034EC0025A40225A90225AE0225B30225B8022582
:0734FC00BD0225C20225C735
:1025CD009006CBE0FE9006CCE0D39E404B9006CA21
:1025DD00E0B404189006CCE0C395725002D231904D
:1025ED0006CBE0D395724002C231802A9006CBE033
:1025FD00C3957250099006CCE0D3957250028002BB
:10260D00D2319006CBE0D3957250099006CCE0C341
:10261D0095725002C231802A9006CBE0D39572405C
:10262D00099006CCE0C3957240028002C23190063B
:10263D00CBE0C3957240099006CCE0D39572400271
:10264D00D231229006CEE0903503F8282873804CC5
:10265D0085527280479000C2E0855EF0A4FFAEF017
:10266D0074081200398F728033856072802E8566F2
:10267D007280298567728024856872801F856972D2
:10268D00801A856A728015856572801085647280E6
:0C269D000B856B728006900016E0F57251
:1035030002265B02265D02266202267602267B02E3
:10351300268002268502268A02268F022694022608
:073523009902269E0226A377
:1026A9009006CFE0FE9006D0E0D39E404B9006CE38
:1026B900E0B404189006D0E0C395725002D232906B
:1026C90006CFE0D395724002C232802A9006CFE04D
:1026D900C3957250099006D0E0D3957250028002DA
:1026E900D2329006CFE0D3957250099006D0E0C35C
:1026F90095725002C232802A9006CFE0D39572407B
:10270900099006D0E0C3957240028002C232900659
:10271900CFE0C3957240099006D0E0D3957240028C
:10272900D232229006D2E090352AF8282873804CBC
:1027390085527280479000C2E0855EF0A4FFAEF03A
:1027490074081200398F728033856072802E856615
:102759007280298567728024856872801F856972F5
:10276900801A856A72801585657280108564728009
:0C2779000B856B728006900016E0F57274
:10352A0002273702273902273E022752022757026B
:10353A00275C02276102276602276B02277002278F
:07354A007502277A02277FBA
:102785009006D3E0FE9006D4E0D39E404B9006D24F
:10279500E0B404189006D4E0C395725002D2339089
:1027A50006D3E0D395724002C233802A9006D3E067
:1027B500C3957250099006D4E0D3957250028002F9
:1027C500D2339006D3E0D3957250099006D4E0C376
:1027D50095725002C233802A9006D3E0D395724099
:1027E500099006D4E0C3957240028002C233900678
:1027F500D3E0C3957240099006D4E0D395724002A8
:10280500D233229006D6E0903551F8282873804CB3
:1028150085527280479000C2E0855EF0A4FFAEF05D
:1028250074081200398F728033856072802E856638
:102835007280298567728024856872801F85697218
:10284500801A856A7280158565728010856472802C
:0C2855000B856B728006900016E0F57297
:1035510002281302281502281A02282E02283302F3
:10356100283802283D02284202284702284C022816
:073571005102285602285BFD
:102861009006D7E0FE9006D8E0D39E404B9006D666
:10287100E0B404189006D8E0C395725002D23490A7
:1028810006D7E0D395724002C234802A9006D7E081
:10289100C3957250099006D8E0D395725002800218
:1028A100D2349006D7E0D3957250099006D8E0C390
:1028B10095725002C234802A9006D7E0D3957240B7
:1028C100099006D8E0C3957240028002C234900696
:1028D100D7E0C3957240099006D8E0D395724002C3
:1028E100D234229006DAE0903578F8282873804CAB
:1028F10085527280479000C2E0855EF0A4FFAEF081
:1029010074081200398F728033856072802E85665B
:102911007280298567728024856872801F8569723B
:10292100801A856A7280158565728010856472804F
:0C2931000B856B728006900016E0F572BA
:103578000228EF0228F10228F602290A02290F027E
:10358800291402291902291E02292302292802299D
:073598002D02293202293740
:10293D009006DBE0FE9006DCE0D39E404B9006DA7D
:10294D00E0B404189006DCE0C395725002D23590C5
:10295D0006DBE0D395724002C235802A9006DBE09B
:10296D00C3957250099006DCE0D395725002800237
:10297D00D2359006DBE0D3957250099006DCE0C3AA
:10298D0095725002C235802A9006DBE0D3957240D5
:10299D00099006DCE0C3957240028002C2359006B4
:1029AD00DBE0C3957240099006DCE0D395724002DE
:1029BD00D23522AE2EAF2F74F5D39F74019E4008F1
:1029CD00782E125F7C022ADA752F01752E00AE511A
:1029DD00AF52E546BE000DD39F40099000A4E0D351
:1029ED00954740028023754700E546C39552F57221
:1029FD009000A7E0D395454008E5452572F5458043
:102A0D00069000A7E0F54580020547900080E0D3D1
:102A1D009560401CE55EC3955F4015AE51AF52E524
:102A2D0046BE00039F50099000A5E0D39548400293
:102A3D00806E9007BCE0A851B80004955250037504
:102A4D004A009007BCE0A851B8000BD39552400640
:102A5D00E5529007BCF0E54A7041E552C39546F545
:102A6D0072E572D3940540037572059000A6E0C31C
:102A7D0095455007E572C3954540028009E545C36C
:102A8D009572F54580069000A6E0F5459000A6E00C
:102A9D00D3954540069000A6E0F5457548008002A7
:102AAD000548E54A7016900080E0C39560500DE52D
:102ABD00462405A851B8000695524002800F90009B
:102ACD0093E0F545754A0174789007BCF022AE2E5F
:102ADD00AF2F74E9D39F74039E4008782E125F7C4C
:102AED00022C79752F01752E00754532A236402ABC
:102AFD00754519900093E075F002A4FFAEF0E5471F
:102B0D00BE0006D39F4002D2360547754A0374783E
:102B1D009007BCF0754900022C68AE51AF52E546E6
:102B2D006F4E7003022C68E546BE000DD39F400921
:102B3D009000A4E0D395474002800F754700E54A09
:102B4D00C394035003754519800DE546C39552F5A1
:102B5D0072E5472572F547900080E0D39560400EF1
:102B6D009007BCE0A851B80007D395524002800CE5
:102B7D000549900093E0B54903754A00E54AB40351
:102B8D0006A20DB3B34002800A0549E549B43C03E2
:102B9D00754A02E54AB402299007BCE0A851B80075
:102BAD000ED395524009E5529007BCF0754900903F
:102BBD000080E0C39560500975490074789007BC9A
:102BCD00F0E54A705A900080E0D39560401CE55EB8
:102BDD00C3955F4015AE51AF52E546BE00039F5001
:102BED00099000A5E0D3954840028008754800750E
:102BFD00454B8028E552C39546F572E572D3940591
:102C0D004003757205900080E0D395604008E5485B
:102C1D002572F5488006E5482406F548754900E516
:102C2D004A7016900080E0C39560500DE54624056E
:102C3D00A851B80006955240028003754A01E54A35
:102C4D00B401187545190549900093E0B54906750D
:102C5D004A0275490074789007BCF0E54575F00A95
:102C6D00A4FFAEF09007B1EEF0A3EFF022E56E9069
:102C7D00359FF8282873900078E07003022E289075
:102C8D0000AEE0B401028003022D7890003CE0B567
:102C9D005D028003022D757E017F00E5BE125F2867
:102CAD00E5BD2FFF50010E8E598F5A7410125F28FB
:102CBD00900066E08E048F05FF125F189007BDEC43
:102CCD00F0A3EDF0E56A60089000D4E064026002C4
:102CDD0080269000D6E0B4011F9007BDE0FEA3E072
:102CED00FF74E7125F28E56A8E048F05FF125F18E7
:102CFD009007BDECF0A3EDF0900078E0B4022790C2
:102D0D0007BFE0FEA3E0FF9007BDE0FCA3E0FDEFF1
:102D1D002DFDEE3CFC74018C068D071200399007D9
:102D2D00BDEEF0A3EFF09007BDE0FEA3E0FF90072E
:102D3D00BFE0FCA3E0FDEDD39FEC9E4004D23980B3
:102D4D0002B2399007BDE0F8A3E09007BFC8F0A329
:102D5D00C8F09000AAE064016006A239B3B3400246
:102D6D0080069007BEE0F55E022E26D2397E017FE9
:102D7D0000E5BE125F28E5BD2FFF50010E8E598F65
:102D8D005A7410125F28900066E08E048F05FF12B2
:102D9D005F189007BDECF0A3EDF0E56A60089000B8
:102DAD00D4E06402600280269000D6E0B4011F904A
:102DBD0007BDE0FEA3E0FF74E7125F28E56A8E040D
:102DCD008F05FF125F189007BDECF0A3EDF090009A
:102DDD0078E0B402279007BFE0FEA3E0FF9007BDA7
:102DED00E0FCA3E0FDEF2DFDEE3CFC74018C068DA7
:102DFD00071200399007BDEEF0A3EFF09007BDE08C
:102E0D00F8A3E09007BFC8F0A3C8F09000AAE06453
:102E1D000160069007BEE0F55E8003755E009000D0
:102E2D0074E07006756E01022C7A75BB180233F3CF
:102E3D00900074E07003022FC97E017F00E5BE1281
:102E4D005F28E5BD2FFF50010E8E598F5A9000BAA5
:102E5D00E0B4010F7E0F7FFFAC59AD5A125F748E37
:102E6D00598F5A9000DFE0B40245AE59AF5A900029
:102E7D001FE0FCA3E0FDEDD39FEC9E400A90001FE8
:102E8D00E559F0A3E55AF0AE59AF5A900021E0FC98
:102E9D00A3E0FDEFD39DEE9C400A900021E559F093
:102EAD00A3E55AF0AE59AF5A74041200398F6090F1
:102EBD0000DFE0704CAE59AF5A90001FE0FCA3E06C
:102ECD00FDEFD39DEE9C4009125F748E598F5A8091
:102EDD0006755A00755900AE59AF5A7410125F2815
:102EED00900063E08E048F05FF125F188C598D5A88
:102EFD0074FFBC0009D39D4005855A608003756041
:102F0D00FE9000AAE0B401028003022FC7A20DB308
:102F1D00B3500E90007EE0A851B80005D3955250E5
:102F2D0003022FBC90007FE075F019A4FFAEF09066
:102F3D0000C2E08E048F05FF125F189000BBE08584
:102F4D0060F0A4FFAEF074648D028C038E048F05C7
:102F5D00FF125F18EA2DFDEB3CFC8C598D5AE56A8A
:102F6D00600F9000D4E0B402089000D6E0640160D8
:102F7D00028017AE59AF5A74E7125F28E56A8E04C6
:102F8D008F05FF125F188C598D5AAE59AF5A9007A5
:102F9D00BDE0FCA3E0FDEDD39FEC9E4005855A5EA0
:102FAD00800BA239B340069007BEE0F55E800BA200
:102FBD0039B340069007BEE0F55E80037560009062
:102FCD000077E07006756E02022C7A75BB1902331C
:102FDD00F3900077E0700302307EE55DD3955040AD
:102FED000302307C90001DE0FEA3E0FFE564125F5C
:102FFD006C90001DEEF0A3EFF07E017F00E5BE1298
:10300D005F28E5BD2FFF50010E8E598F5A9000E4B9
:10301D00E07013740A125F2874518E048F05FF122D
:10302D005F188D648019AE59AF5A740A125F288FDC
:10303D00048E057E017F95CDCCCD125E168F64E595
:10304D0064D39464400375646490001DE0FEA3E0B6
:10305D00FFE5642FFF50010E90001DEEF0A3EFF081
:10306D0090007BE0048E048F05FF125F188D648045
:10307D00037564329000C7E07006756E03022C7AFA
:10308D0075BB130233F39000C7E0604A7E017F00E9
:10309D00E5BE125F28E5BD2FFF50010E8E598F5AE8
:1030AD0074041200398F659000C9E08565F0A4FDA8
:1030BD00ACF07464FF125F188D659000C8E08565F3
:1030CD00F0A4FFAEF074FF8E048F05FF125F18EDB4
:1030DD00900062F08003756500900075E0700675D4
:1030ED006E04022C7A75BB170233F3900075E0B4B1
:1030FD000102800302318C7E017F00E5BE125F2844
:10310D00E5BD2FFF50010E8E598F5A9007C1E0601B
:10311D00199007C1E01490589412008CE493FC743C
:10312D000193FDEDC39FEC9E400280069007C1E028
:10313D0014F09007C1E0C394B3501DAE59AF5A902F
:10314D0007C1E00490589412008CE493FC74019331
:10315D00FDEFC39DEE9C400280069007C1E004F098
:10316D009007C1E0FE90009BE08E0088F0A4FFAEBA
:10317D00F074648E048F05FF125F188D66800375E1
:10318D006600900076E07006756E05022C7A75BBB0
:10319D00160233F3900076E0B4010280030232355B
:1031AD007E017F00E5BE125F28E5BD2FFF50010EA9
:1031BD008E598F5A9007C2E060199007C2E01490A3
:1031CD0059FE12008CE493FC740193FDEDC39FEC4A
:1031DD009E400280069007C2E014F09007C2E0C343
:1031ED0094B3501DAE59AF5A9007C2E0049059FEEA
:1031FD0012008CE493FC740193FDEFC39DEE9C4093
:10320D000280069007C2E004F09007C2E0FE900035
:10321D00A1E08E0088F0A4FFAEF074648E048F05DB
:10322D00FF125F188D67800375670075BB1F023332
:10323D00F37E017F00E5BE125F28E5BD2FFF500133
:10324D000E8E598F5A7409125F2874E68E048F05FD
:10325D00FF125F188D6990007DE07006756E070294
:10326D002C7A75BB150233F390007DE070030233A9
:10327D008F7E017F00E5BE125F28E5BD2FFF500157
:10328D000E8E598F5A74041200398F6890007DE0AC
:10329D00B401159000D1E08568F0A4FFAEF074077D
:1032AD00120039EF9007B6F090007DE0B402159052
:1032BD0000D1E08568F0A4FFAEF07407120039EF7D
:1032CD009007B5F090007DE0B40302800302338DCA
:1032DD009000BEE070389000D1E0601CE568C394AA
:1032ED00195002D22BE568D394644002C22B900092
:1032FD009DE09007B9F08014E568C394195002D28F
:10330D003AE568D394324002C23AC22B80639000F2
:10331D009DE070349000D1E08568F0A4FFAEF074AC
:10332D00FF8E048F05FF125F18ED9007B9F0AE51B7
:10333D00AF52741EBE0006D39F4002D22BE560D360
:10334D0094E54002C22B8029E568C3940A500DAE66
:10335D0051AF52741EBE0004D39F50028002D22B77
:10336D00E560D394E54002C22B90009DE09007B933
:10337D00F09007B9E0C39405500674059007B9F0B5
:10338D0080037568009000D4E07006756E08022CFD
:10339D007A75BB1480509000D4E060397E017F00B7
:1033AD00E5BE125F28E5BD2FFF50010E8E598F5AD5
:1033BD00EFD39421EE940E4005756AFF8015AE593A
:1033CD00AF5A7410125F2874E38E048F05FF125FDD
:1033DD00188D6A8003756A00900078E0600575BBF2
:0633ED001A800375BB18F5
:10359F00022C83022E3D022FDE0230930230F802FE
:0B35AF0031A102323E0232750233A34C
:0533F300056ED2EC2282
:095F5A002582F582500205832224
:0F008C0025E050020583258250020583F582226C
:105EF700EF2F500205832582F582E5833E2EF58339
:015F07002277
:105F6C00CFC39FFF50011E22C3EF9DFFEE9CFE226C
:085F7C000806B6000218062217
:0D5F3600A3E004F07006120049E004F02220
:0E003900048007C3CE13CECF13CFD5E0F6223E
:105E1600BC000FBE0008ED8FF084FFADF022E4FE5B
:105E2600FF22BE000DEF60FE54F0606F20E7030214
:105E36005ECCEAC0E0EBC0E078017A0075F001EED6
:105E460020E710EF25E0FFEE33FE0AC5F023C5F08C
:105E560030E7F0EA5407F9096A7A007B0060010826
:105E6600C3EC9E40167004ED9F4010ED9FFDEC9E26
:105E7600FCE5F0CA4ACA03F5F08005E5F003F5F043
:105E8600C3EE13FEEF13FFD9D77908CACBCAD8D011
:105E9600EAFEEBFFD0E0FBD0E0FA22EC8FF084FCC8
:105EA600ED54F045F0C48FF084FEEDC454F045F097
:105EB600C48FF084FDEEC4FE54F02DFFEE540F3C6B
:105EC600FEADF07C0022790078008FF0EC7E082091
:105ED600E70DC3CD33CD33C933C9C833C8DEF0842B
:105EE60049F9E5F08FF0BE00E6FD7C00E9FFE8FE2B
:015EF6002289
:0E5F2800F88FF0A4FFE5F0CE88F0A42EFE2244
:10000300EF8DF0A4F9A8F0EF8CF0A428F8EE8DF0B2
:06001300A428FEE9FF2213
:105F0800600D782B025F12007830D8FED5E0F822B9
:105F1800EEC0E07E00125E16EFFDEEFCD0E0FE2241
:0C5F4300EEC0E07E00125E16D0E0FE22F0
:03001B0002001EC2
:0300530002005652
:03009B00020071EF
:03000000025F6339
:095F630075817475D000023CDF69
:0B5F4F00E5822FF582E5833EF58322FA
:0A0049000582D5820215831582227C
:10001E00C0E0C0F0C083C082C0D075D000123C19C1
:0B002E00D0D0D082D083D0F0D0E032E0
:10005600C0E0C0F0C083C082C0D075D000123C1C86
:10006600D0D0D082D083D0F0D0E032C0E0C0F0C093
:1000760083C082C0D075D000123CA1D0D0D082D02F
:0600860083D0F0D0E0324F
:00000001FF
